:020000020000FC
:0200000009C035
:1000120098C10CE007BB00EF08BB00E004BB00EF97
:1000220005BB02E001BB0DEF02BB04E00EBF0FE512
:100032000DBF7727002700BD09E109B908E10AB918
:100042000EE800BD05E003BF0EEF402E02BF09B768
:10005200016009BF05E106B978940CEF202EE9D0C2
:1000620032D031D030D02FD045D03DD489D106D432
:100072001DD000E2022149F001E0032131F0DD2729
:10008200CFEF0881051509F414C610D0D2D004D0E0
:1000920052D0C7D07CD1F9CF0F93022D007111F04D
:1000A2000EEF01C00CEF402E0F9108950F9303B392
:1000B20000730695069506950695202E00B30C73DF
:1000C200202A0F9108950F930DE00CD00AE00AD078
:1000D2000F9108950F9306D00D3011F40AE002D06B
:1000E2000F9108955D9BFECF0CB908955F9BFECFE3
:1000F2000CB10895EF93FF93F1E0E6E0CDD3FF91C9
:10010200EF9108950A0D0A0D6D6F726265636F6E4D
:1001120030353032313941200A0D0000EF93FF9320
:10012200C895002021F0002D4CD03196F9CFFF91D7
:10013200EF9177D008950F9301E443D000E02AD0E5
:10014200A1D0022D0C700C30E9F00F9300E239D0EF
:1001520002E437D001E01ED095D00F91043091F027
:100162000F9300E22ED003E42CD002E013D08AD009
:100172000F91083039F000E224D004E422D003E0E9
:1001820009D080D000E21DD00AE01BD00DE019D0CA
:100192000F9108950F93379A0370006407B9369A46
:1001A200349BFECF349AC4B1D5B10F91089501307A
:1001B20039F08894079510F020D0F9CF25D0F7CFE9
:1001C2000895E5D0EF93FF930F9384DF0F910032F0
:1001D20011F427D00FC00B350AF00F750A3252F016
:1001E200F3E0E2E10A52E00F0027F01FC895002D6C
:1001F200DEDF13D0FF91EF9108957260C39A37D07A
:100202007D7FC39834D008957260C39A30D02FD0C6
:100212002ED07D7FC3982BD0089529D028D027D007
:10022200089525D024D023D022D021D020D01FD091
:1002320008950F93022D0370003029F400E00BBDE6
:100242000BEB0ABD12C0013029F403E00BBD09EA31
:100252000ABD0BC0023029F402E10BBD03E40ABD62
:1002620004C001E00BBD04ED0ABD0F9108950F9388
:100272000DE00EBD08B704FFFDCF08BF00E00EBDC4
:100282000F9108950F93112722273327CC2319F4B6
:10029200DD2309F408C0219709EE100F01E0201FA9
:1002A2000027301FF3CF4427552766274395105A5E
:1002B20026483140D8F700EA100F06E8201F01E077
:1002C200301F4A955395105127423040D8F700E12C
:1002D200100F07E2201F00E0301F5A956395185E49
:1002E2002340304078F708EE100F03E0201F00E0B3
:1002F200301F6A95405D042F64DF505D052F61DF7A
:10030200605D062F5EDF8DDF8CDF8BDF0F9108953E
:10031200682A735E7A293F3E3C3830202123272FFA
:1003220047553101014C010611150902140B100445
:100332001E0D1207050F161B0A08030C180E191DB5
:1003420013010F930FB70F93042D02BF71FF0FC05C
:10035200BA9A072F01700395017019F4C2987E7F33
:1003620002C0C29A71600F910FBF0F911895BA988F
:10037200000000000000000000000000F4CF18950B
:1003820095DE2ED066D055D3AFD351D408955F9B5E
:1003920008950CB10D3009F0FACFF89494DE93DE93
:1003A200EFDF86D1A3DE8FDE0F75013479F00234E0
:1003B20079F0033479F0043479F0053479F00835B2
:1003C20009F0EBCFADD274D27EDE23CE0C94540270
:1003D2000C9489040C9416050C945A050C9414067A
:1003E200859B01D00895EF93FF93F5E0E2E354D2A9
:1003F200FF91EF910895EF93FF93F4E0E8E04CD280
:10040200FF91EF9108954F46462020200000EF9380
:10041200FF93F4E0E0E240D2FF91EF91089553653B
:100422006C6563742061206368616E6E656C207414
:100432006F20746F67676C65204F4E2F4F464620C2
:100442006F72205820746F2065586974203E2020F6
:10045200000047D000E246DE45DE44DE43DE42DEF7
:1004620041DE40DE3FDE3EDE3DDE3CDE3BDE832D16
:100472008795879510F450D002C00E94FC018795A1
:1004820010F44AD002C00E94FC01879510F444D0B7
:1004920002C00E94FC01879510F43ED002C00E9467
:1004A200FC0111DE0895D5DF0EDEB1DF1FDE0F7510
:1004B200013459F0023461F0033469F0043471F00C
:1004C200083509F0F0CFFFDD68CF02E03026EBCF30
:1004D20004E03026E8CF08E03026E5CF00E1302600
:1004E200E2CFEF93FF93F4E0E4EFD6D1FF91EF91E7
:1004F20008950A0D4368616E6E656C3A20202020D3
:100502004120202020204220202020204320202083
:10051200202044200A0D0000EF93FF93F5E0EAE269
:10052200BBD1FF91EF9108954F4E20202020000073
:100532000A0D4F5054494F4E414C204F50455241A5
:1005420054494F4E20454449544F522E0A0D2A2AEF
:100552002A2A2A2A2A2A2A2A2A2A2A2A2A2A2A2AF9
:100562002A2A2A2A2A2A2A2A2A2A2A2A2A2A2A2AE9
:100572002A2A2A2A2A2A2A2A2A2A2A2A2A2A2A2AD9
:100582002A2A2A2A2A2A2A2A2A2A2A2A2A2A2A2AC9
:100592002A2A0A0D2A2A2A2A202020202020202046
:1005A200205741524E494E473A2050494E20313150
:1005B2002028444950205041434B41474529204976
:1005C200532047524F554E4445442E202020202090
:1005D200202020202A2A2A2A0A0D2A2A2A2A2020F2
:1005E20020204368616E6765732063616E206265D7
:1005F2002073617665642C2062757420616C6C20B6
:10060200736F6674776172652073656C6563746578
:1006120064206F7074696F6E73202A2A2A2A0A0D69
:100622002A2A2A2A202020206172652064697361A7
:10063200626C6564207768696C652070696E203130
:10064200312069732067726F756E6465642E202095
:100652002020202020202020202020202020202098
:100662002A2A2A2A0A0D2A2A2A2A2A2A2A2A2A2A25
:100672002A2A2A2A2A2A2A2A2A2A2A2A2A2A2A2AD8
:100682002A2A2A2A2A2A2A2A2A2A2A2A2A2A2A2AC8
:100692002A2A2A2A2A2A2A2A2A2A2A2A2A2A2A2AB8
:1006A2002A2A2A2A2A2A2A2A2A2A0A0D0A0D000076
:1006B200EF93FF93F6E0E2ECEFD0FF91EF91089514
:1006C2000A0D4F5054494F4E414C204F5045524114
:1006D20054494F4E20454449544F522E0A0D4D6500
:1006E2006E75206F662050726F6772616D6D616208
:1006F2006C65204F7074696F6E730A0D0A0D412E7E
:100702002E2E2E2E2E5475726E20616E616C6F67C6
:10071200206368616E6E656C73206F6E206F72204D
:100722006F6666200A0D422E2E2E2E2E2E456E74D8
:10073200657220612074657874206D6573736167DA
:1007420065200A0D432E2E2E2E2E2E546F67676CB7
:1007520065205465726D696E616C205365747469AD
:100762006E677320656E61626C652F646973616286
:100772006C650A0D442E2E2E2E2E2E536574204D9E
:100782006F72736520436F646520537065656420E2
:100792000A0D452E2E2E2E2E2E546F67676C652065
:1007A200746F6E65206672657175656E637920621D
:1007B20065747765656E2035303020487A20616E29
:1007C200642031206B487A200A0D582E2E2E2E2EB0
:1007D2002E655869742074686973206D656E752082
:1007E200616E642072657475726E20746F206E6F14
:1007F200726D616C206F7065726174696F6E0A0D43
:100802000A0D506C656173652073656C65637420B5
:10081200616E206F7065726174696F6E20627920FB
:10082200747970696E670A0D412C422C432C442C5A
:10083200452C206F7220582E0A0D3E2000000EE338
:1008420051DCD0E0C0EB52DC083071F008830D308F
:1008520051F0C03619F407E045DCF5CFCA950F9385
:1008620039DC0F91F0CF0895C03B19F407E03ADC70
:10087200EACF30DCC3950DE00883E5CFD0E0C0EBD2
:10088200AA270881CA95A3952DDCC03621F0A03590
:1008920011F00D30B1F70895EF93FF93C895002042
:1008A20021F0002D1FDC3196F9CFFF91EF910895D1
:1008B200DD27CEEF3882F3D1DD27CFEF5882F894CF
:1008C200DD27EE27CFEFEFEF0881E199FECFEEBBF8
:1008D200FFBB0DBBE29AE19AC03619F0EA95CA95C0
:1008E200F3CF78940895DD27FF27CFEFEFEFE1995B
:1008F200FECFEEBBFFBBE09A0DB30883C03619F002
:10090200EA95CA95F4CFDD27CEEF3880C8D1089595
:10091200DADB34D0B3DFD7DB58D091DF0C94CE01D1
:10092200EF93FF93F9E0E2E3B7DFFF91EF910895D0
:100932000A0D0A0D506C6561736520776169742038
:1009420061626F75742032207365636F6E64732CFD
:10095200206E6F772073746F72696E67207365748F
:10096200757020706172616D657465727320696E55
:1009720020454550524F4D2E0A0D0000EF93FF9334
:10098200F9E0EEE889DFFF91EF9108955468652060
:100992006C696E652062656C6F7720636F6E74613F
:1009A200696E73207468652063757272656E746C0B
:1009B200792073746F7265642074657874206D6534
:1009C2007373616765200A0D0000EF93FF93F9E0EE
:1009D200ECED62DFFF91EF910895506C65617365F4
:1009E20020656E7465722074657874206D6573730A
:1009F20061676520746F2062652073746F7265642D
:100A02002E200A0D4D6178696D756D203830206396
:100A1200686172616374657273206F6E206F6E65B8
:100A2200206C696E652E0A0D000001E030260C94E0
:100A3200CE01032D017011F003D008951DD0089549
:100A4200EF93FF93FAE0E2E527DFFF91EF9108953C
:100A52004F7074696F6E73207365742062792074AD
:100A620065726D696E616C2061726520454E41420E
:100A72004C45442E0A0D0000EF93FF93FAE0EAE89A
:100A82000BDFFF91EF9108954F7074696F6E7320C1
:100A9200736574206279207465726D696E616C2071
:100AA2006172652044495341424C45442E200A0D4F
:100AB20000001AD00FE930224BD018DB0F7512DB81
:100AC200013439F0023441F0033449F0043451F076
:100AD200F3CF00E4302A06C000E2302A03C000E669
:100AE200302A00C0F0DA59CC1AD0032D0076003635
:100AF20049F0003461F0003269F002E3F3DA05E311
:100B0200F1DA0BC001E3EEDA00E3ECDA06C001E34E
:100B1200E9DA03C005E3E6DA00C0D5DA0895EF9317
:100B2200FF93FBE0E0E3B8DEFF91EF910895436F9E
:100B3200646520537065656420696E20576F726426
:100B42007320506572204D696E7574653A200000FD
:100B5200EF93FF93FBE0E2E69FDEFF91EF910895B2
:100B62000A0D456E74657220746865206C65747434
:100B72006572207468617420636F72726573706F3E
:100B82006E647320746F207468650A0D636F646508
:100B920020737065656420646573697265642E20D4
:100BA2000A0D412E2E2E2E3120576F726420506571
:100BB20072204D696E7574650A0D422E2E2E2E35E9
:100BC20020576F72647320506572204D696E757480
:100BD20065200A0D432E2E2E2E313020576F72645F
:100BE2007320506572204D696E7574650A0D442E2E
:100BF2002E2E2E323520576F72647320506572206C
:100C02004D696E7574650A0D0A0D506C65617365E8
:100C120020656E74657220412C422C432C6F722029
:100C220044203E20000000E830260C94CE01032D23
:100C3200007811F003D0089519D00895EF93FF932F
:100C4200FCE0EEE429DEFF91EF910895546F6E65AA
:100C5200206F7574707574206973207365742074C5
:100C62006F2031206B487A2E0A0D0000EF93FF931C
:100C7200FCE0EEE711DEFF91EF910895546F6E658F
:100C8200206F757470757420697320736574207495
:100C92006F2035303020487A2E200A0D000055246E
:100CA200DD27CEEF0881500EC03611F0CA95FACF7B
:100CB2000895FCD907D0BDDAEFD919D02AD067DB65
:100CC20059D0FBCFC32DC078C695C695C695032DC6
:100CD2000076069506950695069506950C2B0F93BC
:100CE200022D0C7E202E0F910229202E0895EBD981
:100CF20098DAD0E0C0EBAA270881CA95A39561DAF9
:100D0200C03631F0A03521F00D30B1F78ADA89DA38
:100D120008950F93032D027039F001E452DA00E0D6
:100D220039DAB0DA00E24DDA032D047039F002E468
:100D320048DA01E02FDAA6DA00E243DA032D08707E
:100D420039F003E43EDA02E025DA9CDA00E239DA2D
:100D5200032D007139F004E434DA03E01BDA92DA8D
:100D620000E22FDA00E22DDA0AE02BDA0DE029DACE
:0E0D72000F9108950AE055DA0A95E9F7089501
:00000001FF
